:1000000014360002001E021AF9FFFFFFFFFF023341
:100010001DFFFFFFFFFFFFFFFFFFFFFFFFFF02339B
:10002000C87581CE90FDE88583A012353CEC4D600B
:100030007378AB8003760018B89CFA787F800376DB
:100040000018B865FA78208003760018B820FA788E
:10005000208003760018B81FFA90FDDDAE83AF82D2
:1000600090FBF81200AA6005E4F0A380F690FDE88A
:10007000A88290FDE8A982E8696005E4F20880F7AB
:100080009001081200B390010C1200B390011012FD
:1000900000B39001141200D190011A1200D1900106
:1000A000201200D175D00012341A020126EF6582A9
:1000B0007003EE658322E493F8740193F97402935C
:1000C000FE740393F5828E83E869700122E493F64F
:1000D000A30880F4E493FC740193FD740293FE740E
:1000E0000393FF740493F8740593F58288831200D8
:1000F000AA700122E493A3A883A9828C838D82F045
:10010000A3AC83AD828883898280E32121049B8014
:1001100080049BACAE049BFDE8049D049DFBF304AE
:10012000A2049DFBF30502050280FED0F030F00929
:1001300020F303F68010F7800D30F10920F303F26D
:100140008004F38001F020F404FCD0E0CC22CCC089
:10015000E0120163020154BC0005D0F0ACF022C3F0
:1001600013DCFC02012ABF0009ED258275F001F8BD
:10017000E622BF010FED2582F582EE3583F583750A
:10018000F004E022ED258275F002F8E222D083D05F
:1001900082F5F0C3E493A3C5F095F0C0E0C3D0F0BE
:1001A000E493A395F04012A3A3C3E5F033500205F6
:1001B000832582F58250020583740193C0E0E493A5
:1001C000C0E022D083D082F5F0E4937009740193EB
:1001D0007004A3A3800C74029365F06005A3A3A32D
:1001E00080E7740193C0E0E493C0E022120264024D
:1001F00001FB1202B80201FB1202DC0201FB30E03B
:100200000720E302E622E72230E10720E302E222B0
:10021000E32230E202E022E493221202DC02022313
:100220001202B8020223ABF012022DCBC5F0CB2292
:1002300030E01020E306E6F5F008E622E7F5F009E5
:10024000E7192230E11020E306E2F5F008E222E3AC
:10025000F5F009E3192230E206E0F5F0A3E022E42C
:1002600093F5F074019322BB0003740922BB0107CC
:1002700089828A83740422BB020789828A8374106C
:1002800022740A22020284BB0007E92582F8740165
:1002900022BB010DE92582F582EA3583F5837404DA
:1002A00022BB020DE92582F582EA3583F5837410BD
:1002B00022E92582F87402220202B8BF0005EDF897
:1002C000740122BF01078D828E83740422BF02074E
:1002D0008D828E83741022EDF87402220202DCBF3C
:1002E0000007ED2582F8740122BF010DED2582F58E
:1002F00082EE3583F583740422BF020DED2582F56D
:1003000082EE3583F583741022ED2582F874022283
:10031000020310C0E0120264020328C0E01202B817
:10032000020328C0E01202DC02032830E00B20E3C5
:1003300004D0E0F622D0E0F72230E10B20E304D035
:10034000E0F222D0E0F322D0E0F022C9CDC9CACE3B
:10035000CACBCFCB12035BEDF9EEFAEFFB22BB0069
:100360002FBF000AFAEDF8E7F60809DAFA22BF0112
:10037000128D828E83F802037809A3E7F0D8FA225F
:10038000020383FAEDF8E7F20809DAFA2202038D94
:10039000BB014DBF001489828A83F9EDF802039FE7
:1003A00008A3E0F6D9FA220203B0BF01228D828EA3
:1003B00083FB08C9C582C9CAC583CAE0A3C9C5826F
:1003C000C9CAC583CAF0A3DBEAD8E8220203D38DE9
:1003D000828E83F9EDF8E0F208A3D9FA220203DD58
:1003E000BB024DBF001289828A83F9EDF80203EF48
:1003F00008A3E493F6D9F922BF01238D828E83FBF3
:1004000008C9C582C9CAC583CAE493A3C9C582C93C
:10041000CAC583CAF0A3DBE9D8E722020422898295
:100420008A83F9EDF8E493F208A3D9F922020433A0
:10043000BF000DFAEDF8E3F60809DAFA2202043DEE
:10044000BF01128D828E83F802044A09A3E3F0D81B
:10045000FA22020455FAEDF8E3F20809DAFA220268
:10046000045FE6FB08E6FA08E6F904F618700106F0
:1004700022E6FF08E6FE08E6FD22EFF0A3EEF0A379
:10048000EDF022EBF0A3EAF0A3E9F022E0FFA3E015
:10049000FEA3E0FD22E0FBA3E0FAA3E0F9220000C6
:1004A00000000000000502006105710026059800AB
:1004B000330A0900610A750066154400610CF900F1
:1004C0006109A9006109E000610DC000610BF10044
:1004D000610A1C00610A510061173C0033174F008C
:1004E000341E1400431EBF0044202C0044201A0078
:1004F000471EE600471F8B004D1FDC004F1F080002
:100500005832A800617CCC7DFF121CC52290FFFCF4
:10051000E020E72DC2AFAE59AF58755A20E55A1406
:10052000C55A6019E4FE7F05EE4FCE24FFCECF34CE
:10053000FFCF6007E490FF92F080ED80E08E598F4E
:10054000582212050A7D077CB71232C47D0F7C6EDB
:100550001232DE789D7A06E4F608DAFC7A06120595
:10056000CD7C03120E55122168E4FEFF7C0F12327F
:100570004DD2A822123138E490FC38F090FFF0E020
:1005800030E408740190FC39F08005E490FC39F007
:100590007D0A7C001225461231BB2212313890FCB4
:1005A00039E014700E90FFF0E04410F07C0012254A
:1005B000DF801990FC39E0700E90FFF0E054EFF00E
:1005C0007C001225DF80057C171225DF1231BB224B
:1005D00090FFF0E054ABF090FFF0E04420F0228C6C
:1005E000378D367882EDF608ECF6EDFEECFD7F01F6
:1005F0009000051201F57880F67882E6FD08E6FCA9
:10060000EDFEECFD7F019000041201F5540FFC7D1E
:100610008012176D7880E6700DAD3AAE39AF38E4D0
:100620001203187C082290FFF0E054FEF090FFF0D7
:10063000E054FDF0801E7882E6FD08E6FCEDFEEC5D
:10064000FD7F0190000812021725E0440190FFF39E
:10065000F00206D97882E6FD08E6FCEDFEECFD7FAF
:100660000190000612021754FE90FFF3F0802B78E1
:1006700082E6FD08E6FCEDFEECFD7F01900008122D
:100680000217FAEB90FFF1F01208C8400DAD3AAE38
:1006900039AF38E41203187C18227882E6FD08E6A8
:1006A000FCEDFEECFD7F0190000812021790FFF1B7
:1006B000F01208C8400DAD3AAE39AF38E412031855
:1006C0007C18227882E6FD08E6FCEDFEECFD7F0159
:1006D000900006120217440190FFF3F07883E6249D
:1006E00003F618E63400F67880E624FE500990FF01
:1006F000F0E054FDF0800790FFF0E04402F0E49059
:10070000FFF1F0788176007880E624FFFCE434FF86
:10071000FD7881E67F00FEECD39EEF6480CD64809F
:100720009D402F1208AD400F7881E6AD3AAE39AF4B
:10073000381203187C182290FFF2E0FC788286833E
:10074000088682ECF0788106A37882A68308A682C8
:1007500080B51208AD400F7881E6AD3AAE39AF38BA
:100760001203187C182290FFF2E0FC78828683083E
:100770008682ECF07880E6AD3AAE39AF38120318D5
:100780007C00228C378D367882EDF608ECF6EDFE93
:10079000ECFD7F019000051201F57881F67882E684
:1007A000FD08E6FCEDFEECFD7F019000041201F572
:1007B000540FFC7D8112176D7881E670037C08224E
:1007C00090FFF0E054FEF090FFF0E054FDF0801B4D
:1007D0007882E6FD08E6FCEDFEECFD7F0190000866
:1007E00012021725E090FFF3F0805B7882E6FD08A7
:1007F000E6FCEDFEECFD7F0190000612021754FEB0
:1008000090FFF3F080217882E6FD08E6FCEDFEEC37
:10081000FD7F01900008120217FAEB90FFF1F01231
:1008200008C840037C18227882E6FD08E6FCEDFE4D
:10083000ECFD7F0190000812021790FFF1F0120802
:10084000C840037C18227883E6240AF618E63400B0
:10085000F6788076007881E624FFFCE434FFFD78AA
:1008600080E67F00FEECD39EEF6480CD64809D40E7
:100870002178828683088682E090FFF1F01208C812
:1008800040037C1822788006788306E618700106FB
:1008900080C390FFF0E04401F0788286830886826E
:1008A000E090FFF1F01208C840037C18227C00227F
:1008B00090FFF0E020E71290FFF0E030E50990FFB4
:1008C000F0E04420F0C32280E7D32290FFF0E02044
:1008D000E31290FFF0E030E50990FFF0E04420F0F3
:1008E000C32280E7D3228C428D417C00ED54F0FD81
:1008F000EC7003ED64307005753E038003753E04B3
:10090000AC3E120F72758300858340E541540FF5AC
:100910003FE5407004E53F64037035E53E24FD7516
:10092000F00AA42402F582E434FCF583E030E60505
:100930001210598019E53E249DF8E654FBF678A97B
:10094000E62405F58218E63400F583740FF080592B
:10095000E5407004E53F64047048E53E24FD75F011
:100960000AA42402F582E434FCF583E030E507AC08
:1009700042AD41121C5AE54230E21578ADE630E056
:100980000F78ADE630E109E4FF04FE7C0412324D3D
:1009900078A9E62406F58218E63400F583740FF092
:1009A0008007E4FC7DEE121C5AC203221231381279
:1009B0000F7278A9E62406F58218E63400F583E084
:1009C00090FC38F078A9E62405F58218E63400F5A5
:1009D00083E090FC39F0C2037D027C0012254612B0
:1009E00031BB221231387895ECF6EC249DF8E630D4
:1009F000E1077C131225DF800F90FC39E0FD78952C
:100A0000E6FC1213EF1225DF1231BB2212313878C7
:100A100095ECF67D00120F121225DF1231BB221267
:100A200031387895ECF6EC249DF8E630E2077C133B
:100A30001225DF801B7895E6249DF8E620E1077CEF
:100A4000121225DF800A7895E6FC1214131225DFB6
:100A50001231BB221231387895ECF6EC249DF8E681
:100A600020E2077C111225DF800A7895E6FC12153A
:100A7000141225DF1231BB221231387895ECF612B0
:100A80000F7278A9E62409F58218E63400F583E0B0
:100A900090FC3FF078A9E6240AF58218E63400F5C8
:100AA00083E090FC40F078A9E62403F58218E63450
:100AB00000F583E0FC78A9E62404F58218E634000A
:100AC000F583E0F56278A9E62402F58218E63400A1
:100AD000F583E0F5638C61E4EC333354017895F6EB
:100AE0006008E56230E1037895067895E690FC4170
:100AF000F078A7E62402F58218E63400F583E0FDDD
:100B0000A3E0540CFCED54E68C65F564E56130E53A
:100B100003436501E56220E50EE561547F7008E559
:100B20006120E703436502E56130E303436510E5B7
:100B30006130E203436520E561540360034365408F
:100B4000E56130E103436580E56130E4034364011E
:100B5000E56130E603436408E56220E40EE5615494
:100B60007F7008E56120E7034364105365FB53641D
:100B7000F9AD64E56590FC3ACDF0A3CDF0E56330C6
:100B8000E30DE5635430C4540F90FC3DF08005E460
:100B900090FC3DF0E563540390FC3CF0E5635404A5
:100BA000C31390FC3EF090FC3CE0700E7D357EFC63
:100BB0007F01740190000912014B78A9E62408F521
:100BC0008218E63400F583E07C00FD78A9E624076E
:100BD000F58218E63400F583E07F004CFEEF4D907F
:100BE000FC38F0A3CEF0CEC2037D0A7C001225466D
:100BF0001231BB221231387895ECF6789A760108DA
:100C000076FC0876387897760C789A12046E120281
:100C10001D7898CBF6CB08F67F00EF24EA401FE45E
:100C2000EF25E090357EFD93CD04937899667003AF
:100C3000ED186670067897760080030F80DC789652
:100C4000EFF6789A12046E9000021202177898CB91
:100C5000F6CB08F65404CB54064B60047897760B19
:100C60007899E630E313789A12046E900005120129
:100C7000F524FB50047897760D7899E654C07D00F2
:100C800064C04D70047897760B789A12046E9000C9
:100C9000041201F524FC50047897760F789A120418
:100CA0006E9000061201F524FD50047897760E78B8
:100CB0009A12046E9000091201F524FD50047897F1
:100CC000760A7897E6702A7895E6FC120F72789A81
:100CD00012046E78A7E6F978A6E6FA7B01740A7822
:100CE00000120348C2037895E6FC1211157897ECC0
:100CF000F67897E6FC1225DF1231BB2212313878E4
:100D000095ECF6120F727895E624FD75F00AA4248E
:100D100014F582E434FCF583AC82AD8378A6868337
:100D2000088682ECF9EDFA7B0A78011203B0C2035F
:100D30007895E6FC1211151231BB228D2B8C2AED11
:100D400060407527017529487528FFE52A24FDFCB8
:100D5000E434FFFDEC7C0325E0CD33CDDCF9FCE58C
:100D6000292CF529E5283DF528AD29AE28AF2774B3
:100D7000809000061203207480900002120320125B
:100D80000FC5E52B14603B7527017529087528FFF1
:100D9000E52A24FDFCE434FFFDEC7C0325E0CD33A3
:100DA000CDDCF9FCE5292CF529E5283DF528AD2910
:100DB000AE28AF27E4900006120320E49000021250
:100DC0000320221231387895ECF6EC249DF8E630B9
:100DD000E2097895E6FC121514D2007895E6FC122B
:100DE0000F727896760090FC39E030E704789676BA
:100DF000017896E6FD7895E6FC120D38C2033000C6
:100E0000077895E6FC1214137C001225DF1231BB23
:100E10002278A9E62404F58218E63400F583E0443C
:100E200001F078A9E62404F58218E63400F583E0A1
:100E300030E00280ED78A9E6240BF58218E6340054
:100E4000F583E054F8F078A9E62402F58218E63438
:100E500000F583E04480F022C2038C58120F7278B0
:100E6000A6868308868279AF7A357B0A78011203D9
:100E7000FE120E0EAC587D02120D38C203AC581291
:100E80001115228D538E528F518C50120F72754F47
:100E90000078A9E62405F58218E63400F583E02001
:100EA000E41FE54F24F64019054FC2037C181232A7
:100EB000FB90FF93E04401F0B2B3AC50120F72808C
:100EC000D078A9E62405F58218E63400F583E02001
:100ED000E405C2037C022278A9E62405F58218E61F
:100EE0003400F583E0540F601678A9E62405F582F6
:100EF00018E63400F583E0540FF0C2037C01227839
:100F0000A88683088682E0AD53AE52AF5112031813
:100F1000C2037C00228D318C30121514E531600F34
:100F2000E530B4030A7C0112250E7C8112250EAC3B
:100F300030120F72E531601A78AA8683088682E043
:100F400054E7F0A3A3A3A3E054E7F0AC307D021272
:100F50000D3878A6868308868279B97A357B0A7837
:100F6000011203FEC203E530249DF8E654FDF6AC01
:100F700030121115228C2630030512329A80F87C2B
:100F80000A1231ADD203E52624FD78A3F670077866
:100F9000AA76FF0876E078A3E67D007C0425E0CD04
:100FA00033CDDCF9FC24A078A9F6ED34FF18F678EF
:100FB000A3E675F00AA42400FCE434FCFD78A6ED59
:100FC000F608ECF61232462278A9E62402F58218D9
:100FD000E63400F583E030E72278A9E62402F582C2
:100FE00018E63400F583E0547FF078A9E62402F592
:100FF0008218E63400F583E04480F02278AA8683E4
:10100000088682E0547FF0AD83E5822404FCE43D51
:101010008C82F583E0547FF078A9E6240BF58218E2
:10102000E63400F583E054F8F078ABE62401F5826D
:1010300018E63400F583E04403F078ABE62405F5C8
:101040008218E63400F583E04403F078A9E624052D
:10105000F58218E63400F583740FF02278AA8683AF
:10106000088682E0543FF0AD83E5822404FCE43D31
:101070008C82F583E0543FF078A3E624A4F8E6FCE4
:1010800078ABE62401F58218E63400F583ECF078BD
:10109000A3E624A4F8E6FC78ABE62405F58218E67E
:1010A0003400F583ECF078A9E6240BF58218E634D9
:1010B00000F583E054FB4402F52678A7E62402F508
:1010C0008218E63400F583E030E50343260178A971
:1010D000E62405F58218E63400F583E030E00312DB
:1010E0000FC5E526FC78A9E6240BF58218E6340046
:1010F000F583ECF078A9E62405F58218E63400F5CE
:1011000083740FF078AA8683088682E04480F0A377
:10111000A3A3A3E04480F0228C2A120F7278A7E6E2
:101120002408F58218E63400F583E0FC78A9E6246B
:101130000AF58218E63400F583ECF078A7E6240778
:10114000F58218E63400F583E0FC78A9E62409F579
:101150008218E63400F583ECF078A6868308868250
:10116000E0FDA3E0FCEDFE78A9E62408F58218E690
:101170003400F583EEF0ECFE78A9E62407F582183A
:10118000E63400F583EEF08C298D28C3EC9405ED50
:10119000940C400575277C8033D3E5299401E5281C
:1011A0009403400575273C8023D3E5299481E528E5
:1011B000940140057527188013D3E5299460E5282C
:1011C0009400400575270C8003752708AF27E4EFCE
:1011D000547C4483FF8F27E527FC78ABE62401F598
:1011E0008218E63400F583ECF0E527FC78ABE624C2
:1011F00005F58218E63400F583ECF0E527FC78A3CA
:10120000E624A4F8ECF678A9E62402F58218E63480
:1012100000F583E0F52778A7E62402F58218E63486
:1012200000F583A3E030E3175327C778A7E624052A
:10123000F58218E63400F583E09035AA93422778CA
:10124000A7E62402F58218E63400F583E030E705CE
:1012500043274080035327BF5327FB78A7E6240684
:10126000F58218E63400F583E06003432704532732
:10127000FC78A7E62404F58218E63400F583E04202
:1012800027432780E527FC78A9E62402F58218E6A3
:101290003400F583ECF078A9E62404F58218E634EE
:1012A00000F583E0F52778A7E62402F58218E634F6
:1012B00000F583A3E030E1055327DF8003432720B7
:1012C00078A7E62402F58218E63400F583E030E4DE
:1012D000055327EF800343271078A7E62409F582FA
:1012E00018E63400F583E0B40203432702E527FC47
:1012F00078A9E62404F58218E63400F583ECF0784A
:10130000A9E62403F58218E63400F583E0F5277892
:10131000A7E62409F58218E63400F583E07005534A
:10132000277F800343278078A7E62402F58218E60A
:101330003400F583A3E030E00543272080035327E2
:10134000DF78A7E62402F58218E63400F583E03062
:10135000E30543274080035327BF78A7E62402F51F
:101360008218E63400F583E030E00543271080035F
:101370005327EF78A7E62402F58218E63400F583B8
:10138000A3E030E40543270880035327F778A7E656
:101390002402F58218E63400F583A3E030E5054326
:1013A000270480035327FB78A7E62402F58218E67A
:1013B0003400F583A3E030E605432701800353277B
:1013C000FE78A7E62402F58218E63400F583A3E050
:1013D00030E70543270280035327FDE527FC78A962
:1013E000E62403F58218E63400F583ECF0C2037CB2
:1013F00000228D278C26ED54031460037C1022E517
:1014000027547C24FC40037C0B22E526249DF8E62F
:101410004402F67C00228C30120F72E530249DF8D5
:10142000E620E24FAC307D02120D38E53024FE4458
:1014300028FC78AA8683088682ECF0AF83E58224B4
:1014400004FEE43FFFEC8E828F83F07C038C2CE55E
:101450002CFC78ABE62401F58218E63400F583EC29
:10146000F0E52CFC78ABE62405F58218E63400F5AF
:1014700083ECF0752D01752F48752EFFE53024FDA6
:10148000FCE434FFFDEC7C0325E0CD33CDDCF9FC3E
:10149000E52F2CF52FE52E3DF52E78ABE62404F54F
:1014A0008218E63400F583E054E7F52CAD2FAE2E1C
:1014B000AF2DE4900002120320E4900006120320F6
:1014C0001201EF30E503432C10E52CFC78ABE62449
:1014D00004F58218E63400F583ECF012105978A96F
:1014E000E62406F58218E63400F583E0C203FCE545
:1014F00030249DF8E64404F68C2CE530540FC45497
:10150000F07E00FFEEEF44047D00FFEC4EFCED4F5B
:10151000FD121CC57C00228C2F120F72120FF9785D
:10152000AA8683088682E05408F0A3A3A3A3E0540C
:1015300008F0AC2F7D02120D38C203E52F249DF870
:10154000E654FBF67C00221231387896ECF6EC2457
:101550009DF8E630E10A7D007C131225461231BB6E
:101560007896E6249DF8E64401F67896E6FC120F9C
:10157000727896E624FD75F00AA42414F582E4340A
:10158000FCF58378A6E6FA08E6F97B0A78011203EF
:10159000B078A6868308868279B97A357B0A780185
:1015A0001203FE120FC5C2037896E6FC12111578DD
:1015B00095ECF6EC600A7D007C081225461231BBE2
:1015C0007896E6FC120F7278A9E62404F58218E6F4
:1015D0003400F583E0441054DFFC78A9E62404F5D8
:1015E0008218E63400F583ECF07895ECF6C2037CC3
:1015F000C81232FB7896E6FC120F7278A9E6240432
:10160000F58218E63400F583E054EFF0C2037CC89D
:101610001232FB7896E6FC120F7278A9E62404F5E4
:101620008218E63400F583E04410F0C2037CC8124F
:1016300032FB7896E6FC120F7278A9E62404F58254
:1016400018E63400F583E04420F0C2037CF0123247
:10165000FB7896E6FC120F7278A9E62405F582184D
:10166000E63400F583E030E415C2037896E64410D2
:101670007F00FE7C0712324D1231BB02173B78A966
:10168000E62404F58218E63400F583E054CFF0C276
:10169000037CC81232FB7896E6FC120F7278A9E63A
:1016A0002404F58218E63400F583E04430F0C203E8
:1016B0007CF01232FB7896E6FC120F7278A9E624D1
:1016C00005F58218E63400F583E030E414C20378AF
:1016D00096E644107F00FE7C0712324D1231BB802B
:1016E0005D78A9E62404F58218E63400F583E05419
:1016F000EFF078A9E62404F58218E63400F583E0DB
:1017000054DFF07896E624FD75F00AA42414F582DF
:10171000E434FCF583AC82AD8378A68683088682A8
:10172000ECF9EDFA7B0A78011203B0C2037896E671
:10173000FC1211157D007C0B1225461231BB2212C2
:101740003138E490FC39F07D027C001225461231DC
:10175000BB221231387C001225DF1231BB22743CCF
:1017600090FBE0F0743E90FBE0F0E490FC28F02267
:101770008D358C34ECB401028003D340028028B450
:1017800002028003D34008A835E625E0F68018B4AD
:1017900004028003D3400AA835E625E025E0F68060
:1017A00006A83576008000228C3C8D3BEDFEECFDDA
:1017B0007F0175660675670090FC29120477120197
:1017C000EFB480028006D3500302186E90FC2912F9
:1017D00004899000031201F554F0B430028003D361
:1017E000405F90FC29120489900008120217FAFD4C
:1017F000EBFE7F0190FC2C120477EECD9035C3FCFC
:10180000E493FF740193FEF9EFFA7B01EAFFE9FE2E
:10181000ECC39EED9F40259035C5E493FD74019384
:10182000FCEDFEECFD7F01EECDFC90FC2EE0D39CA8
:1018300090FC2DE09D5005756680803312198C80D8
:101840002EB460028003D3400BAC3CAD3B1207804A
:101850008C66801BB41003B34010C3B42003B340A4
:1018600009C3B440028003D34000756681800080C4
:1018700075B481028003D3406B90FC2912048990D7
:1018800000031201F554F0B430028003D3401D90E0
:10189000FC29120489900008120217FAFDEBFE7F62
:1018A0000190FC2F1204771218F68036B460028083
:1018B00003D34013753A67E4F539F538AC3CAD3BDA
:1018C0001205DC8C66801BB41003B34010C3B42037
:1018D00003B34009C3B440028003D340007566815E
:1018E000800080028000E566FC90FC29120489ECEF
:1018F000900002120320AC672290FC291204899008
:1019000000041201F5600474018001E4A2E0920178
:1019100090FC29120489ED2403FD50010E90FC2C4B
:1019200012047790FC291204899000051201F5F544
:10193000679000041201F5540FFC7D6712176DE5E6
:10194000677004756608227566007884760078846E
:10195000E6C39567503890FC2F1204891201EFFC02
:1019600090FC2C120489EC12031830010E90FC310B
:10197000E004F090FC307003E004F078840690FC02
:101980002EE004F090FC2D7003E004F080C0229063
:10199000FC2AE0FDA3E0FCEDFEECFD7F01ED240A56
:1019A000FD50010E90FC3212047790FC291204893C
:1019B0009000041201F5540FB401028003D34017C4
:1019C00090FC321204890DED70010E90FC2F120470
:1019D0007778887601804EB402028003D340199054
:1019E000FC32120489ED2402FD50010E90FC2F12EE
:1019F000047778887602802DB404028003D34019DE
:101A000090FC32120489ED2404FD50010E90FC2F4D
:101A100012047778887604800CB400028003D340E7
:101A2000007566082290FC291204899000051201B5
:101A3000F5F567788576007885E6C39567400302FB
:101A40001AF4788676007886E6C378889650769081
:101A5000FC2C1204891201EFFC90FC321204921249
:101A600001E9F45CFC1201E9F890FC2F120489E80A
:101A7000C0E01201EFC8D0E0C8584CFC90FC2C121A
:101A80000489EC1203187887ECF690FC31E004F03E
:101A900090FC307003E004F009E970010A90FC3218
:101AA00012048090FC291204899000041201F53080
:101AB000E40E90FC2EE004F090FC2D7003E004F0A6
:101AC00078860680817888E6FDE4FEFFEECDFC9006
:101AD000FC31E02CF090FC30E03DF07888E6FDE44D
:101AE000FEFFEECDFC90FC34E02CF090FC33E03DAA
:101AF000F0788506021A347566002222C0E0C0F034
:101B0000C082C083C0D0E8C0E0E9C0E0EAC0E0EB3A
:101B1000C0E0ECC0E0EDC0E0EEC0E0EFC0E090FF60
:101B200092E01201C01B47301B47321B56381B681E
:101B30003A1B7A3E1B92441B86461B9E501BE0526A
:101B40001BBF541C015600001C2290FF92E07F0036
:101B5000FE7C0112324D021C32E4FF04FE7C0312B3
:101B6000324D742090FFFEF0021C32E4FF04FE7C34
:101B70000212324D744090FFFEF0021C32E4FF046A
:101B8000FE7C0412324D021C32E4FF04FE7C05127E
:101B9000324D021C32E4FF04FE7C0612324D021C60
:101BA0003290FFA5E07D0090FBF8CDF0A3CDF09042
:101BB000FBF9E0FCF58390FBF8E04433FD121CC513
:101BC000807390FFB5E07D0090FBFACDF0A3CDF0DF
:101BD00090FBFBE0FCF58390FBFAE04443FD121C14
:101BE000C5805290FFA6E07D0090FBFCCDF0A3CD18
:101BF000F090FBFDE0FCF58390FBFCE04434FD122B
:101C00001CC5803190FFB6E07D0090FBFECDF0A3B7
:101C1000CDF090FBFFE0FCF58390FBFEE04444FD3B
:101C2000121CC5801090FF92E07D00FCED44AAFDDF
:101C3000121CC58000E490FF92F0D0E0FFD0E0FEDF
:101C4000D0E0FDD0E0FCD0E0FBD0E0FAD0E0F9D06D
:101C5000E0F8D0D0D083D082D0F0D0E0320581053A
:101C60008105810581A881181818EDF608ECF69019
:101C7000FF5AE020E70280F790FF59E07D00A8813D
:101C800018CDF6CD08F67D03A881E618FCE6CC2534
:101C9000E0CC33CCDDF9CCF6CC08F6A88118E644CC
:101CA000F8F6A881181818E6FD08E6FCA881188641
:101CB00083088682EDF0A3ECF0740290FF5AF015D1
:101CC0008115811581158122E5812405F581E4A81E
:101CD0008118F6A88118181818EDF608ECF690FB94
:101CE000F5E024F85003021DE6E4A8811818F6A8D0
:101CF0008118E6FEA88118181818E6FD08E6FC7F92
:101D000000EF24F8404DE4EF25E0247DF582E43433
:101D1000FCF583E0FBA3E06C7003FAEB6D700974D3
:101D200001A8811818F6802BE4EF25E0247DF582C8
:101D3000E434FCF5837A00E054F0CCF8CCCDF9CD56
:101D4000FB7800E954F0F9EA687002EB6970010E63
:101D50000F80AEA88118EEF6A88118181818EDF6B5
:101D600008ECF6A881EFF6A8811818E67079A8812A
:101D700018E624F74071A88118181818E6540FA81F
:101D800081F664046017A881E664036010A88118D6
:101D9000181818E6FD08E6FC121C5A804A7C0A1244
:101DA00031ADA88118181818E6FD08E6FC90FBF480
:101DB000E025E0247DF582E434FCF583EDF0A3EC2E
:101DC000F090FBF4E0FFE4EF045407FF90FBF4F025
:101DD00090FBF5E004F012324690FBF6E07008E468
:101DE000FEFF7C0F12324D802790FBF7E004F05489
:101DF0003F701D90FBF7E044FE7D00FC90FBF4E09B
:101E000025E0247DF582E434FCF583EDF0A3ECF0CD
:101E1000E58124FBF58122788B7600788C7600743E
:101E20000190FBF6F012313890FBF5E060577C0A28
:101E30001231AD90FBF3E025E0247DF582E434FC23
:101E4000F583E0FDA3E0FC90FBF3E025E0247DF5C5
:101E500082E434FCF583E4F0A3F090FBF3E0FFE4CC
:101E6000EF045407FF90FBF3F090FBF5E014F078DB
:101E700089EDF608ECF61232467889E6FD08E6FCB4
:101E80001208E380A312329A90FF93E04401F0B26B
:101E9000B3788B06B60011788B7600788CE6F40464
:101EA00004A2E092B4788CF6021E25E490FBF6F0D2
:101EB00090FBF5E07D00FCED44CFFD121C5A123181
:101EC000BB22123138E5706449456F601590FF837D
:101ED000E0540F7D00D39570ED956F5005122F8162
:101EE00080031230511231BB22123138E57064493F
:101EF000456F600512308B800E90FF80E04408F043
:101F000090FF83E0547FF01231BB221231388C54A1
:101F1000EC54F0B41015756A357569FC756801E507
:101F20006A2403F56AE5693400F569E4F557F55666
:101F3000E556C394015027E554540FFCAD6AAE69D1
:101F4000AF68120E808C55EC60028012056AE56A5B
:101F5000700205690557E5577002055680D2E554B1
:101F6000540F249DF8E654FEF6E554540F7F00FE0E
:101F70007C1212324DE5551470097D007C09122542
:101F8000468007AD577C001225461231BB22123124
:101F90003890FFFCE04402F090FF00E030E713903F
:101FA000FF83E04480F0436D8090FFFCE04401F04B
:101FB000801190FF82E04408F0536D7F90FFFCE0B9
:101FC00054FEF090FF81E04480F01225F990FFFE6E
:101FD000E04405F090FFFCE054FDF01231BB22120A
:101FE00031387C011232FB78ADE64402F674FEFC17
:101FF00004FD121CC590FF5AE030E70280F7E4F5BB
:102000004E754D10AC4EAD4DE54E154E7002154D52
:10201000EC4D600280EE4387011231BB2212313851
:102020007C021231C778ADE654FDF61231BB2212A4
:10203000313878ADE630E02C78ADE630E12678AD89
:10204000E6FCF58318E644F0FD121C5A90FFFCE014
:102050004420F07C021232FB78ADE654FDF6741A8F
:1020600090FFFEF078ADE6FCF58318E644F1FD1232
:102070001C5A1231BB22756D0090FFFFE0600343D4
:102080006D01756E00E4F56CF56BE4F56F757049E4
:10209000748490FF82F0748490FF80F0748090FFCD
:1020A00058F0748090FF5AF0AD46AF457E00EE24A4
:1020B000FE5003022142E4EE75F007A4247FF5826E
:1020C000E434F8F583E0FFE4EF5480FDE4EF540FCF
:1020D00014FFED6038E4EF75F008A42448F582E4BD
:1020E00034FFF5837490F0E4EF75F008A4244AF50A
:1020F00082E434FFF5837480F0E4EF75F008A424E3
:102100004EF582E434FFF5837480F08034E4EF759B
:10211000F008A42408F582E434FFF5837490F0E419
:10212000EF75F008A4240AF582E434FFF583E4F0A7
:10213000E4EF75F008A4240EF582E434FFF583E49F
:10214000F00E0220AB8D468E448F45747F90FFFDCC
:10215000F0749090FFFCF0228C58EC24F65006E5C9
:10216000582437FC22E5582430FC22D2B0122543F3
:10217000EC700302227E755C03AE5B7F00E55C15AC
:102180005C6480247F5035EF2400F582E434FBF555
:1021900083E0FE24FE501EEF7D00FCE4FB7474C35C
:1021A0009CFAEB9DFBEE7D00FCEAC39CED6480CBCA
:1021B00064809B50028005EF2EFF80C18E5B8F5A9A
:1021C000E55C6480247F500302227EE55A248E5011
:1021D0000302227E855A5D755B00AE5AAF5B903577
:1021E000EEE493F55CE55C155C6480247F5018EEAA
:1021F0002400F582E434FBF583E0FCEF9035EE93A8
:102200006C70040E0F80DE8E5A8F5BE55C64802458
:102210007F406E755E017560E8755FFFE55D2402C5
:10222000F55A755C07E55C334057AD60AE5FAF5E55
:10223000E55CF5823395E0F5831201F5C4540FFC9B
:10224000122155E55A2400F582E434FBF583ECF0C5
:10225000055A055AAD60AE5FAF5EE55CF582339519
:10226000E0F5831201F5540FFC122155E55A2400C4
:10227000F582E434FBF583ECF0055A055A155C80D1
:10228000A4740290F851F090F86B79C77A357B27E7
:1022900078011203FE756A357569FC756801E49072
:1022A000FF83F0748090FF81F0755902E55975F055
:1022B00007A4247FF582E434F8F583E0788FF6FCF8
:1022C000540F14FC788FECF6E55975F007A42481BF
:1022D000F582E434F8F583E0789276FD0876E8FC40
:1022E000788FE675F008A42448F582E434FFF5837E
:1022F000E4F0788FE675F008A4244FF582E434FF0B
:10230000F583ECF07892E6FF08E67E03CFC313CFA7
:1023100013DEF9FE788FE675F008A42449F582E40F
:1023200034FFF583EEF0788FE675F008A4244AF5C3
:1023300082E434FFF5837480F07890ECF67D0078C9
:1023400093E62CF618E63DF67892E6FD08E67C0367
:10235000CDC313CD13DCF9FC788FE675F008A42407
:102360004DF582E434FFF583ECF0788FE675F008E4
:10237000A4244EF582E434FFF583E4F07892E6FD80
:1023800008E6FC788FE6FF7E00EE24FE5003022470
:10239000FDE4EE75F007A4247FF582E434F8F583BC
:1023A000E0FFE4EF5480FAE4EF540F14FFE4EE751D
:1023B000F007A42481F582E434F8F583E07890F600
:1023C000E4EE1313548024F0F8E434FDF9E8FCE95A
:1023D000FD8A5AEA700302246AE4EF75F008A42427
:1023E00048F582E434FFF583E4F07890E6FAE4EF10
:1023F00075F008A4244FF582E434FFF583EAF0ED8C
:10240000FBEC7A03CBC313CB13DAF9FAE4EF75F0E4
:1024100008A42449F582E434FFF583EAF07890E6D5
:102420007B00FAEC2AFCED3BFDFBEC7A03CBC313FB
:10243000CB13DAF9FAE4EF75F008A4244DF582E441
:1024400034FFF583EAF0E4EF75F008A4244AF5823E
:10245000E434FFF5837480F0E4EF75F008A4244EB3
:10246000F582E434FFF5837480F00224F9E4EF751B
:10247000F008A42408F582E434FFF583E4F07890B2
:10248000E6FAE4EF75F008A4240FF582E434FFF5D2
:1024900083EAF0EDFBEC7A03CBC313CB13DAF9FA42
:1024A000E4EF75F008A42409F582E434FFF583EA2B
:1024B000F07890E67B00FAEC2AFCED3BFDFBEC7A31
:1024C00003CBC313CB13DAF9FAE4EF75F008A424B5
:1024D0000DF582E434FFF583EAF0E4EF75F008A42B
:1024E000240AF582E434FFF583E4F0E4EF75F008A4
:1024F000A4240EF582E434FFF583E4F00E02238673
:102500008E597892EDF608ECF6788FEFF61220737C
:10251000228C26EC30E718E526540F1475F008A439
:102520002448F582E434FFF583E054DFF08016E5BB
:1025300026540F1475F008A42408F582E434FFF53E
:1025400083E054DFF0227C0022EC90FC37F08C24F6
:10255000ED2403F5257D00D39572ED95714003853B
:102560007225E52524B75009752503740290FC37C0
:10257000F0AC2512307622E4F56CF56B12257D2245
:1025800090FC35E06573600E740490FC37F0E4F560
:102590006B756C0380467D73E4FEFF79357AFC7BB6
:1025A0000174057800120348E56C2403F56CE56BB3
:1025B0003400F56BE56CD39572E56B95714006853B
:1025C000726C85716BD3E56C9448E56B9400400C9C
:1025D000740290FC37F0E4F56B756C03AC6C123050
:1025E0007622EC90FC37F0E4F56CF56B8C32EC6005
:1025F0000512306780057C001230762290FF93E050
:102600004401F0B2B390FF04E0F54A90FF06E0FD0C
:10261000A3E0ED7D00FC7D00FC90FF06E0FFA3E061
:102620007E00FFE4FEEC4EFCED4FFDC3EC9448ED64
:102630009400502290FF06E0FDA3E0ED7D00FC7DBC
:1026400000FC90FF06E0FFA3E07E00FFE4FEEC4EFE
:10265000FCED4FFD8004E4FD7C488C728D7190FF91
:1026600002E0FDA3E0ED7D00FC7D00FC90FF02E0B8
:10267000FFA3E07E00FFE4FEEC4EF54CED4FF54B82
:10268000756A357569FC7568017D357EFC7F017959
:1026900073E4FAFB74057800120348754900E549B4
:1026A00024FE4019AD6AAE69AF68E412031805490B
:1026B0000DED70010E8D6A8E698F6880E1756A3547
:1026C0007569FC75680190FF00E05460B4000280F9
:1026D00006D35003022CBFE54A540FF549E54A548E
:1026E00080A2E0920290FF01E012018A000B2CBA56
:1026F000270528232CBA292F2CBA2A122A462BADBB
:102700002BB02BF02C632C91E56D30E70EE54C459A
:102710004B7008E572640245716003022CBC90FFA7
:1027200000E0541FB400028003D34029E54A60034F
:10273000022820AD6AAE69AF68740112031878AD43
:10274000E630E00BAD6AAE69AF6874021203187C24
:102750000212307622B401028003D3401BE56D20C3
:10276000E107E54A6003022820E54A24FE500302FF
:1027700028207C0212307622B402028006D3500355
:1027800002281EE56D20E10DE54A6009E54A6480F6
:102790006003022820AC4A1230FD4003022820E5E5
:1027A00049702530021190FF80E05408AD6AAE698F
:1027B000AF68120318800F90FF82E05408AD6AAE34
:1027C00069AF68120318803D154930021DE549754F
:1027D000F008A42448F582E434FFF583E05408AD02
:1027E0006AAE69AF68120318801BE54975F008A44A
:1027F0002408F582E434FFF583E05408AD6AAE693D
:10280000AF68120318AD6AAE69AF681201EF600BD2
:10281000AD6AAE69AF6874011203187C021230769B
:10282000228000022CBCE56D20E706E57245716050
:1028300003022CBC90FF00E0541FB400028003D3BD
:10284000401AE54C14454B7004E54A600302292CFC
:1028500078ADE654FEF67C0012307622B401028098
:1028600003D3402AE56D20E108E56D20E00302294D
:102870002CE56D30E004E54A700BE56D30E109E5CB
:102880004A24FE500302292C7C0012307622B40226
:10289000028006D3500302292AE54C454B6003020F
:1028A000292CAC4A1230FD400302292CE56D20E1B1
:1028B00007E56D20E0028077E56D30E006E54960D0
:1028C00002806CE549700F90FF82E054F7F090FFB2
:1028D00080E054F7F022E549B401028003D34009B7
:1028E0007D017C03120F128011B402028003D340D9
:1028F000097D017C04120F1280001549300215E594
:102900004975F008A42448F582E434FFF583E054C7
:10291000F7F08013E54975F008A42408F582E43443
:10292000FFF583E054F7F07C00123076228000023D
:102930002CBCE56D20E706E57245716003022CBCF6
:1029400090FF00E0541FB400028003D3401AE54C0E
:1029500014454B7004E54A6003022A0F78ADE64443
:1029600001F67C0012307622B401028003D34029A4
:10297000E56D20E108E56D20E003022A0FE56D30EA
:10298000E004E549700BE56D30E108E54924FE50AF
:1029900002807F7C0012307622B402028003D34092
:1029A0006FE54C454B60028069AC4A1230FD400235
:1029B0008060E56D20E107E56D20E0028054E54987
:1029C000701430020990FF80E04408F0800790FF07
:1029D00082E04408F022E56D30E1331549300215FC
:1029E000E54975F008A42448F582E434FFF583E056
:1029F0004408F08013E54975F008A42408F582E442
:102A000034FFF583E04408F07C0012307622800227
:102A10008000022CBCE56D20E712E5724571700C58
:102A2000E54A700890FF00E0541F6003022CBCE5EB
:102A30004C90FFFFF090FFFFE06005436D018003C5
:102A4000536DFE7C0012307622E56D30E70EE572A4
:102A50004571600890FF00E0541F6003022CBCAD7C
:102A60004BE54CED7D00FC7D00FCBD0002800302C7
:102A70002BA8B401028003D34032E54A7005E54C2F
:102A8000FC6003022BAA756A407569F8756801D36A
:102A9000E5729412E57194004006E4FD7C12800416
:102AA000AC72AD718C708D6F12308B22B4020280CB
:102AB00003D34059E54A6003022BAAE54CFC70277A
:102AC000756A527569F8756801D3E5729419E571F4
:102AD00094004006E4FD7C198004AC72AD718C70EA
:102AE0008D6F12308B8025756A6B7569F87568017A
:102AF000D3E5729427E57194004006E4FD7C2780BD
:102B000004AC72AD718C708D6F12308B22B40302E5
:102B10008006D35003022BA8E54CF549700F90FFB7
:102B200004E0FDA3E04D6003022BAA801890FB0295
:102B3000E0FDA3E0FC90FF05E06C700790FF04E06F
:102B40006D60028068E4F570F56F7F00E54914C59B
:102B500049600FEF2400F582E434FBF583E02FFF9A
:102B600080EA8F4AE54A2400F582E434FBF583E0ED
:102B70007D00D39572ED95714006AC72AD71800FFA
:102B8000E54A2400F582E434FBF583E07D00FC8C0B
:102B9000708D6FE54A2400FCE434FBFDFEECFD7F04
:102BA000018D6A8E698F6812308B228000022CBCE6
:102BB000022CBCE56D30E719E5721445717012E521
:102BC0004A700EE54C454B700890FF00E0541F60C2
:102BD00003022CBCE56D20E008E56D20E103022C2A
:102BE000BC756A6EE4F569F568E4F56F04F570127A
:102BF000308B22E56D20E727E57245717021E54AAB
:102C0000701DE54C6402454B600DE54C14454B606E
:102C100006E54C454B700890FF00E0541F6003022E
:102C20002CBCE56D20E008E56D20E103022CBC859D
:102C30004C6EE56E700A436D01536DFDD2B080207D
:102C4000E56E64026007E56E1460028072536DFEEB
:102C5000436D02E56E64026005E56E147002C2B059
:102C60007C0012307622E56D30E71AE5721445716A
:102C70007013E54A700FE54C454B700990FF00E07A
:102C8000541F1460028038E56D20E10280317C0120
:102C900012307622E56D20E715E5724571700FE57B
:102CA0004C454B700990FF00E0541F146002800FE8
:102CB000E56D20E10280087C00123076228000025F
:102CC0002F7DB440028006D35003022F7390FF0182
:102CD000E090FC35F0E54A90FC36F0E490FC37F0EB
:102CE000E56A2403F56AE5693400F569AD4BE54C06
:102CF000856A82856983CDF0A3CDF090FF01E01253
:102D000001C02D2A012D50022D7A032DA4042DF28D
:102D1000052E2F062E55072E7B082EA7092ECD0B2C
:102D20002EF30C2F02802F028100002F60E56D2012
:102D3000E7067C051225DF227D767E357F02793815
:102D40007AFC7B01740878001203487D087C00122D
:102D5000254622E56D20E7067C051225DF22E54A9F
:102D6000B403004010B40500500BE54A7F00FE7C20
:102D70001012324D227D007C0712254622E56D207F
:102D8000E7067C051225DF22E54AB403004010B4B3
:102D90000500500BE54A7F00FE7C1112324D227D6A
:102DA000007C0712254622E56D20E7067C051225EA
:102DB000DF22E54AB405028003D3400AE4FF04FEA3
:102DC0007C0A12324D22B401028003D3400AE4FF90
:102DD00004FE7C0812324D22B403004010B40500FA
:102DE000500BE54A7F00FE7C1312324D227D007CA1
:102DF0000712254622E56D20E734D3E5729448E5B5
:102E00007194005006E572457170067C021225DF50
:102E100022E54AB40103B3400BC3B403004009B434
:102E200006005004123123227C071225DF221225CE
:102E30007D22E56D20E71DE54AB403004010B4058E
:102E400000500BE54A7F00FE7C1612324D227C07B3
:102E50001225DF2212257D22E56D20E71DE54AB40B
:102E600003004010B40500500BE54A7F00FE7C19BA
:102E700012324D227C071225DF2212257D22E56DBC
:102E800020E723748190FF93F0E54AB403004010DB
:102E9000B40500500BE54A7F00FE7C1712324D222C
:102EA0007C071225DF2212257D22E56D20E71DE536
:102EB0004AB403004010B40500500BE54A7F00FE01
:102EC0007C1812324D227C071225DF2212257D222A
:102ED000E56D20E71DE54AB403004010B40500503D
:102EE0000BE54A7F00FE7C1512324D227C0712252D
:102EF000DF2212257D22E56D20E7067C071225DF03
:102F00002212257D22E56D30E72090FF00E0541F5E
:102F1000701090FF01E0B480051225748003122523
:102F20007D227D007C051225462290FF00E0541F83
:102F300060067C051225DF22D3E5729448E5719482
:102F400000500BC3E5729407E571940050067C03B2
:102F50001225DF22E54AB40504123123227C071230
:102F600025DF22E56D30E7087D007C05122546222D
:102F70007C051225DF22B420028003D340008000AC
:102F80001230512275430090FF83E0540FD39543D4
:102F90004024E54324F0F582E434FEF583E0AD6A95
:102FA000AE69AF6812031805430DED70010E8D6A0E
:102FB0008E698F6880D1E5437D00FCC3E5709CF588
:102FC00070E56F9DF56FE570456F6006E490FF83D7
:102FD000F02290FF82E04408F0E4F56F75704990AC
:102FE000FC35E0B405028003D3404090FC36E0F5A8
:102FF00043B405028003D3400AE4FF04FE7C0B12B5
:10300000324D22B401028003D3400AE4FF04FE7C67
:103010000912324D22B403004010B40500500BE5F4
:10302000437F00FE7C1412324D2222B480004023E4
:10303000B48200501E7C357DFC1217A57D008C6C7F
:103040008D6B90FC37E0600512305180057C0012DA
:103050003076222290FF83E0547FF090FF82E0449C
:1030600008F090FF80E04408F02290FF82E04408DE
:10307000F090FF80E04408F0228C237D008C708D5E
:103080006F756A357569FC75680112308B2290FF87
:1030900083E0547FF0E5706449456F700122C3E519
:1030A000709408E56F94004015752108E5217D00B6
:1030B000FCC3E5709CF570E56F9DF56F8009857028
:1030C00021E4F56F757049752200E522C395215002
:1030D00026AD6AAE69AF681201EFFCE52224F8F56F
:1030E00082E434FEF583ECF005220DED70010E8DC7
:1030F0006A8E698F6880D3E521547F90FF81F0222A
:103100008C487F00EF24FD4019E4EF75F007A424FC
:103110007FF582E434F8F583E065487002D3220F2E
:1031200080E28F47C32285727085716F90FF82E0C5
:1031300054F7F090FF83E0547FF022C000C001C03C
:1031400002C006C007E5782408F8860653067F7C8F
:10315000FF1231AD7C007D00E57B6046FF90FD9560
:10316000E0547F6E700FC083C082A3E0FDA3E0FC3B
:10317000A3157B8007A3A3A3DFE68026DF06D0820A
:10318000D083801EE0F8A3E0F9A3E0FAD082D083D8
:10319000E8F0A3E9F0A3EAF0A3C083C082A3A3A34D
:1031A00080DA123246D007D006D002D001D00022F9
:1031B00085A87A75A888EC70027C3F8C7922E57826
:1031C0002408F8760012329A80FBC000C001C002C9
:1031D000C006C007AE047CFF1231ADE57B6042FF44
:1031E00090FD95E0547F6E700BC083C082A3A3A3B3
:1031F000157B8007A3A3A3DFEA8026DF06D082D059
:103200008380D8E0F8A3E0F9A3E0FAD082D083E885
:10321000F0A3E9F0A3EAF0A3C083C082A3A3A38034
:10322000DA7808087918097C01E6547F6E70067612
:10323000007700800608090CBC08EE123246D00761
:10324000D006D002D001D00022757900857AA8225C
:10325000C0F0C082C083C3E57B24E8500512329AD7
:1032600080F4EC6031903575E493C39C4028C00431
:103270007CFF1231ADD004430480E57B75F003A4DC
:103280002495F582E434FDF583ECF0EFA3F0EEA392
:10329000F0057B123246D083D082D0F022C0047C6D
:1032A00020D28CD28DD504FDD0042275A80075885B
:1032B0000075B80075F00075D000E4F8900000F6D5
:1032C00008B800FB020000C3ED940250047D037CAB
:1032D000E8ECF4FCEDF4FD0CBC00010D8C7F8D7E60
:1032E00022C3EC94BCED940250047D077CD0ECF436
:1032F000FCEDF4FD0CBC00010D8C7D8D7C22EC708E
:103300000122C000E5782418F8A604E5782408F81E
:10331000C6547FF6E630E703D0002212329A80F4DA
:10332000C28C857C8C857D8AD28CC0E0C0D0C0F0F8
:10333000C082C083C000C001C002C003C004C00579
:10334000C006C007121AF8E5782408F8E66024E5FC
:10335000782410F8A681E57875F021A4248DF582F3
:10336000E434FCF58378AEE58104C398F9E6F0080F
:10337000A3D9FA74082578F8057808E65480700C0B
:10338000E578B407F3780875780080EFE5782410C5
:10339000F88681E57875F021A4248DF582E434FC6B
:1033A000F58378AEE58104C398F9E0F608A3D9FA6D
:1033B000D007D006D005D004D003D002D001D00071
:1033C000D083D082D0F0D0D0D0E032C0E0C0D0C026
:1033D00000C001C002C28E857E8D857F8BD28E7823
:1033E0001979097A07E77004A600800BE6600816D1
:1033F000E67004E74480F70809DAEAE57960131417
:10340000F579700EE5782408F87600123246D28CF1
:10341000D28DD002D001D000D0D0D0E0327581ADB5
:10342000742A90FF93F0757F30757EF8757D607516
:103430007CF012053F1234CE12175B90FF93E044EC
:1034400001F0B2B31234F81232A880DA22C0007C44
:1034500001EC2408F8E660090CBC08F512329A80E9
:10346000EED00022C0F0C082C083C000C006C007FA
:10347000ED2410F876BCED75F021A4248DF582E4DE
:1034800034FCF583C082C083A3A3E4780DF0A3D8F5
:10349000FCEC547F75F002A42441F582E5F034354C
:1034A000F583E493FE740193F5828E83E493FE74B6
:1034B0000193FFD083D082EFF0A3EEF0ED2408F863
:1034C000EC4480F6D007D006D000D083D082D0F074
:1034D00022757800757B007A08791878087600776D
:1034E000000809DAF8E478087480447FF67401442F
:1034F00010F58975B808D2ABD2A9227581ADD28EEC
:10350000D28CD2AFE57B6032FF90FD95E0548060B5
:103510002478087908E0547FFA7B00E6547FB502EE
:10352000027BFF08D9F5EB700CEAF012344AAD04C7
:10353000AC02123461A3A3A3DFD212329A80C57CFD
:10354000017D002204FE04F204F604EA04E604E22B
:1035500004EE04FA04A604AA04D604DA04A204A21F
:1035600004A204DE04BE04B604BA04B204CA04C64B
:1035700004C204CE04D204AE1901030022004802A2
:1035800000480E301420C81AD0180A0C0506020391
:1035900001020001CE0181010000C0008000600036
:1035A0003000180010000800040002000100081894
:1035B00028380C05100A0200000000000301100A60
:1035C000020000000000FBE0FBF2090227000102FC
:1035D00000A0FA0904000003FF00000007058102B3
:1035E00040000007050102400000070583030200B8
:1035F00001220354005500530042003300340031CF
:1036000000300020002000200020002000200020AA
:073610000020000000000093
:00000001FF
